 pwrbtn

 Timestamp is 4da2a511 (Mon Apr 11 18:52:01 2011)

 Preferred load address is 10000000

 Start         Length     Name                   Class
 0001:00000000 000003daH .rdata                  CODE
 0001:000003dc 00000023H .rdata$debug            CODE
 0001:00000400 000009a0H .text                   CODE
 0001:00000da0 00000028H .idata$2                CODE
 0001:00000dc8 00000014H .idata$3                CODE
 0001:00000ddc 0000005cH .idata$4                CODE
 0001:00000e38 00000084H .idata$6                CODE
 0001:00000ec0 000000c8H .edata                  CODE
 0002:00000000 0000005cH .idata$5                DATA
 0003:00000000 00000058H .pdata                  DATA

  Address         Publics by Value              Rva+Base       Lib:Object

 0000:00000000       ___safe_se_handler_count   00000000     <absolute>
 0000:00000000       ___safe_se_handler_table   00000000     <absolute>
 0001:0000001c       ??_C@_1BO@JIEELHHJ@?$AA?9?$AAP?$AAW?$AAR?$AAB?$AAT?$AAN?$AA?5?$AAI?$AAn?$AAi?$AAt?$AA?$AN?$AA?6?$AA?$AA@ 1000101c     pwrbtn.obj
 0001:00000040       ??_C@_1HK@DHAGHLLL@?$AAF?$AAa?$AAt?$AAa?$AAl?$AA?5?$AAE?$AAr?$AAr?$AAo?$AAr?$AA?$CB?$AA?5?$AA?5?$AAF?$AAa?$AAi?$AAl?$AAe?$AAd?$AA?5?$AAt?$AAo?$AA?5?$AAc?$AAr?$AAe?$AAa?$AAt?$AAe?$AA?5?$AAP@ 10001040     pwrbtn.obj
 0001:000000c0       ??_C@_1FM@LPDJHABL@?$AAC?$AAo?$AAu?$AAl?$AAd?$AA?5?$AAn?$AAo?$AAt?$AA?5?$AAi?$AAn?$AAi?$AAt?$AAi?$AAa?$AAl?$AAi?$AAz?$AAe?$AA?5?$AAP?$AAo?$AAw?$AAe?$AAr?$AAB?$AAu?$AAt?$AAt?$AAo?$AAn@ 100010c0     pwrbtn.obj
 0001:00000120       ??_C@_1JC@MPAFOHFI@?$AAE?$AAR?$AAR?$AAO?$AAR?$AA?3?$AA?5?$AAF?$AAa?$AAi?$AAl?$AAe?$AAd?$AA?5?$AAt?$AAo?$AA?5?$AAr?$AAe?$AAq?$AAu?$AAe?$AAs?$AAt?$AA?5?$AAt?$AAh?$AAe?$AA?5?$AAs?$AAy?$AAs@ 10001120     pwrbtn.obj
 0001:000001b4       ??_C@_1DO@NCDJIGLK@?$AAE?$AAR?$AAR?$AAO?$AAR?$AA?3?$AA?5?$AAu?$AAn?$AAa?$AAb?$AAl?$AAe?$AA?5?$AAt?$AAo?$AA?5?$AAc?$AAr?$AAe?$AAa?$AAe?$AA?5?$AAe?$AAv?$AAe?$AAn?$AAt?$AA?$AN?$AA?6?$AA?$AA@ 100011b4     pwrbtn.obj
 0001:000001f4       ??_C@_1BA@BIMMLBCK@?$AAP?$AAi?$AAo?$AAr?$AAi?$AAt?$AAy?$AA?$AA@ 100011f4     pwrbtn.obj
 0001:00000204       ??_C@_1BO@PBJLKMGC@?$AAd?$AAe?$AAb?$AAo?$AAu?$AAn?$AAc?$AAe?$AAP?$AAe?$AAr?$AAi?$AAo?$AAd?$AA?$AA@ 10001204     pwrbtn.obj
 0001:00000228       ??_C@_1FA@JIHAJLLD@?$AAu?$AAn?$AAa?$AAb?$AAl?$AAe?$AA?5?$AAt?$AAo?$AA?5?$AAa?$AAl?$AAl?$AAo?$AAc?$AAa?$AAt?$AAe?$AA?5?$AAm?$AAe?$AAm?$AAo?$AAr?$AAy?$AA?5?$AAf?$AAo?$AAr?$AA?5?$AAc?$AAo@ 10001228     pwrbtn.obj
 0001:00000278       ??_C@_1CI@OHCJFJPM@?$AAE?$AAR?$AAR?$AAO?$AAR?$AA?3?$AA?5?$AA?$CF?$AAs?$AA?5?$AAl?$AAi?$AAn?$AAe?$AA?5?$AA?$CF?$AAd?$AA?3?$AA?5?$AA?$AA@ 10001278     pwrbtn.obj
 0001:000002a0       ??_C@_1JA@BFAGHCDG@?$AAc?$AA?3?$AA?2?$AAw?$AAi?$AAn?$AAc?$AAe?$AAr?$AAo?$AAo?$AAt?$AAs?$AA?2?$AAt?$AAo?$AAp?$AAa?$AAz?$AA?2?$AAw?$AAi?$AAn?$AAc?$AAe?$AA7?$AA0?$AA0?$AA?2?$AAp?$AAl?$AAa@ 100012a0     pwrbtn.obj
 0001:00000330       ??_C@_1BO@BBAGPNEJ@?$AA?$CL?$AAP?$AAW?$AAR?$AAB?$AAT?$AAN?$AA?5?$AAI?$AAn?$AAi?$AAt?$AA?$AN?$AA?6?$AA?$AA@ 10001330     pwrbtn.obj
 0001:00000350       ??_C@_1EC@DKCANKJI@?$AAP?$AAw?$AAr?$AAB?$AAu?$AAt?$AAt?$AAo?$AAn?$AA?5?$AA?3?$AA?5?$AAD?$AAL?$AAL?$AA_?$AAP?$AAR?$AAO?$AAC?$AAE?$AAS?$AAS?$AA_?$AAD?$AAE?$AAT?$AAA?$AAC?$AAH?$AA?$AN?$AA?6@ 10001350     pwrbtn.obj
 0001:00000398       ??_C@_1EC@JGJFBEHA@?$AAP?$AAw?$AAr?$AAB?$AAu?$AAt?$AAt?$AAo?$AAn?$AA?5?$AA?3?$AA?5?$AAD?$AAL?$AAL?$AA_?$AAP?$AAR?$AAO?$AAC?$AAE?$AAS?$AAS?$AA_?$AAA?$AAT?$AAT?$AAA?$AAC?$AAH?$AA?$AN?$AA?6@ 10001398     pwrbtn.obj
 0001:00000400       PwrButtonIntrThread        10001400 f   pwrbtn.obj
 0001:000005e4       PWR_Deinit                 100015e4 f   pwrbtn.obj
 0001:00000738       PWR_Init                   10001738 f   pwrbtn.obj
 0001:00000aec       DllEntry                   10001aec f   pwrbtn.obj
 0001:00000b58       PWR_PowerUp                10001b58 f   pwrbtn.obj
 0001:00000b88       PWR_PowerDown              10001b88 f   pwrbtn.obj
 0001:00000b98       PWR_IOControl              10001b98 f   pwrbtn.obj
 0001:00000bbc       PWR_Open                   10001bbc f   pwrbtn.obj
 0001:00000be0       PWR_Close                  10001be0 f   pwrbtn.obj
 0001:00000c04       GetCurrentThread           10001c04 f i pwrbtn.obj
 0001:00000c1c       SetEvent                   10001c1c f i pwrbtn.obj
 0001:00000c50       SetSystemPowerState        10001c50 f   coredll:COREDLL.dll
 0001:00000c60       InterruptDone              10001c60 f   coredll:COREDLL.dll
 0001:00000c70       WaitForSingleObject        10001c70 f   coredll:COREDLL.dll
 0001:00000c80       CeSetThreadPriority        10001c80 f   coredll:COREDLL.dll
 0001:00000c90       LocalFree                  10001c90 f   coredll:COREDLL.dll
 0001:00000ca0       KernelIoControl            10001ca0 f   coredll:COREDLL.dll
 0001:00000cb0       CloseHandle                10001cb0 f   coredll:COREDLL.dll
 0001:00000cc0       EventModify                10001cc0 f   coredll:COREDLL.dll
 0001:00000cd0       CreateThread               10001cd0 f   coredll:COREDLL.dll
 0001:00000ce0       InterruptInitialize        10001ce0 f   coredll:COREDLL.dll
 0001:00000cf0       CreateEventW               10001cf0 f   coredll:COREDLL.dll
 0001:00000d00       RegQueryValueExW           10001d00 f   coredll:COREDLL.dll
 0001:00000d10       OpenDeviceKey              10001d10 f   coredll:COREDLL.dll
 0001:00000d20       LocalAlloc                 10001d20 f   coredll:COREDLL.dll
 0001:00000d30       NKDbgPrintfW               10001d30 f   coredll:COREDLL.dll
 0001:00000d40       DisableThreadLibraryCalls  10001d40 f   coredll:COREDLL.dll
 0001:00000d50       DDKGpioSetConfig           10001d50 f   cspddk:CSPDDK.dll
 0001:00000d60       DDKGpioReadDataPin         10001d60 f   cspddk:CSPDDK.dll
 0001:00000d70       DDKGpioClearIntrPin        10001d70 f   cspddk:CSPDDK.dll
 0001:00000d80       DDKIomuxSetPadConfig       10001d80 f   cspddk:CSPDDK.dll
 0001:00000d90       DDKIomuxSetPinMux          10001d90 f   cspddk:CSPDDK.dll
 0001:00000da0       __IMPORT_DESCRIPTOR_COREDLL 10001da0     coredll:COREDLL.dll
 0001:00000db4       __IMPORT_DESCRIPTOR_CSPDDK 10001db4     cspddk:CSPDDK.dll
 0001:00000dc8       __NULL_IMPORT_DESCRIPTOR   10001dc8     coredll:COREDLL.dll
 0002:00000000       __imp_SetSystemPowerState  10002000     coredll:COREDLL.dll
 0002:00000004       __imp_InterruptDone        10002004     coredll:COREDLL.dll
 0002:00000008       __imp_WaitForSingleObject  10002008     coredll:COREDLL.dll
 0002:0000000c       __imp_CeSetThreadPriority  1000200c     coredll:COREDLL.dll
 0002:00000010       __imp_LocalFree            10002010     coredll:COREDLL.dll
 0002:00000014       __imp_KernelIoControl      10002014     coredll:COREDLL.dll
 0002:00000018       __imp_CloseHandle          10002018     coredll:COREDLL.dll
 0002:0000001c       __imp_EventModify          1000201c     coredll:COREDLL.dll
 0002:00000020       __imp_CreateThread         10002020     coredll:COREDLL.dll
 0002:00000024       __imp_InterruptInitialize  10002024     coredll:COREDLL.dll
 0002:00000028       __imp_CreateEventW         10002028     coredll:COREDLL.dll
 0002:0000002c       __imp_RegQueryValueExW     1000202c     coredll:COREDLL.dll
 0002:00000030       __imp_OpenDeviceKey        10002030     coredll:COREDLL.dll
 0002:00000034       __imp_LocalAlloc           10002034     coredll:COREDLL.dll
 0002:00000038       __imp_NKDbgPrintfW         10002038     coredll:COREDLL.dll
 0002:0000003c       __imp_DisableThreadLibraryCalls 1000203c     coredll:COREDLL.dll
 0002:00000040       \177COREDLL_NULL_THUNK_DATA 10002040     coredll:COREDLL.dll
 0002:00000044       __imp_DDKGpioReadDataPin   10002044     cspddk:CSPDDK.dll
 0002:00000048       __imp_DDKGpioClearIntrPin  10002048     cspddk:CSPDDK.dll
 0002:0000004c       __imp_DDKIomuxSetPadConfig 1000204c     cspddk:CSPDDK.dll
 0002:00000050       __imp_DDKIomuxSetPinMux    10002050     cspddk:CSPDDK.dll
 0002:00000054       __imp_DDKGpioSetConfig     10002054     cspddk:CSPDDK.dll
 0002:00000058       \177CSPDDK_NULL_THUNK_DATA 10002058     cspddk:CSPDDK.dll

 entry point at        0001:00000aec

 Static symbols

